:107800000C945D3C0C94953C0C947A3C0C947A3C22
:107810000C947A3C0C947A3C0C947A3C0C947A3C10
:107820000C947A3C0C947A3C0C947A3C0C947A3C00
:107830000C947A3C0C947A3C0C947A3C0C947A3CF0
:107840000C947A3C0C947A3C0C947A3C0C947A3CE0
:107850000C947A3C0C947A3C0C947A3C0C947A3CD0
:107860000C947A3C0C947A3C040309041C037700C2
:10787000770077002E0066006900730063006800DF
:107880006C002E00640065000E035500530042009A
:1078900061007300700012011001FF000008C016A3
:1078A000DC05020101020001090212000101008051
:1078B000FA09040000000000000011241FBECFEFF1
:1078C000D8E0DEBFCDBF11E0A0E0B1E0EEE1F0E82E
:1078D00002C005900D92A630B107D9F711E0A6E0DD
:1078E000B1E001C01D92AD33B107E1F70E94B63D92
:1078F0000C940D400C94003CA82FB92F80E090E030
:1079000041E050EA609530E009C02D9182279795BB
:10791000879510F084279527305EC8F36F5FA8F332
:107920000895EADF8D939D930895CF93CFB7CF93BA
:10793000DF93C3954F9BE9F74F9B0BC04F9B09C04B
:107940004F9B07C04F9B05C04F9B03C04F9B01C07F
:1079500089C06F93C0912001DD27C95DDE4F2F9351
:1079600065E54F9B03C02F916F91E6CF0F931F9357
:107970004F9320E040E15F9309B1047807FB27F9BA
:107980003F9350E03BE039C0147840642F77012FDB
:107990005F5F1EC0406819B114782F7752501FC026
:1079A000406409B12F770478D1F15F5F00C023C034
:1079B000406219B12F77147891F15F5F00C025C044
:1079C00004781027515012F45D5F00001150279584
:1079D0002C3F19B1C8F614780127015027952C3F88
:1079E000C8F64227499309B1047810274F73115004
:1079F00027952C3FA8F64695469519B1147879F04D
:107A00000127015027952C3F98F66B5A60F33150AF
:107A100009B1B0F600C011E01CBB002717C03B50F5
:107A20003195C31BD04011E01CBB0881033CF9F029
:107A30000B34E9F020911E011981110F1213EDCFC3
:107A4000093651F10D3211F0013E39F7009325014D
:107A50003F915F914F911F910F912F916F91CCB3F7
:107A6000C0FD67CFDF91CF91CFBFCF911895209107
:107A70002501222369F310912301112339F53430B4
:107A80003AF13093230120931F01109120013BE034
:107A9000311B309320011CC0009123010130B4F44C
:107AA0000AE53091000134FD14C000930001C3E1E8
:107AB000D1E013C0052710E000C000000BB91AC0C8
:107AC000052710E0221F1DC010E021C04AE502C0BA
:107AD00032ED432FC4E1D0E032E01AB114685F9A6E
:107AE0000BB11AB954E820E865E320FF05270BB96C
:107AF000279517951C3FF0F66695B8F7B1F720FF6C
:107B000005270BB9279517951C3FD0F62795179594
:107B100017FF052700001C3F0BB9B0F629913A95D5
:107B200019F70B7710912401110FC651D0400BB9F2
:107B300011F010931E0111E01CBB00681AB11B77F5
:107B4000402F4B7754E05A95F1F70BB91AB94BB95E
:107B50007FCF1BB8F8941DBA1092690081E085BFF1
:107B600015BEE0911101F091120109952F923F92FB
:107B70004F925F926F927F928F929F92AF92BF923D
:107B8000CF92DF92EF92FF920F931F93CF93DF93E9
:107B900088E10FB6F89480936000109260000FBEE9
:107BA0005F9A04B601FE21C214BE81E085BF82E067
:107BB00085BF4F991AC280916900836080936900E4
:107BC000E89A4F9BFECF57987894E8E86E2EE8E746
:107BD0007E2E7CE6472E78E7572E68E6262E68E74D
:107BE000362E58EAC52E58E7D52E46E9A42E48E78A
:107BF000B42E37E0832E31E0932E909123019350E1
:107C000097FD60C1809120012CE0E22EF12CE81A52
:107C1000F10827E231E0E20EF31E80911F018D3260
:107C200009F0D9C0983009F04BC133EC30931301FF
:107C30008AE58093000110920B01D7013C91832FBC
:107C4000807611962C911197882309F452C0909256
:107C5000220180922101233009F513969C911397FC
:107C600014968C91149712962C91203339F48370CA
:107C7000E82FF0E0EE5FFE4F80810CC0203A19F44F
:107C80000E94F73F07C0203C21F4F70165810E9464
:107C9000FF3F80E080930A0194E08AC0253011F410
:107CA00091E086C0822F84508630E0F4D70112968E
:107CB0008D919C91139790930D0180930C01293025
:107CC00009F475C016969C91169790930E0115961F
:107CD0008C91827080930F012093100137FD6EC04C
:107CE0002FEF6DC0223009F062C0B1E0B093060101
:107CF0005EC0F701828110921C01222331F41092A0
:107D00001D012CE131E092E04DC0253019F4809343
:107D1000240145C0263099F5D70113968C91813006
:107D200029F4B0922201A092210106C0823031F4E0
:107D3000D0922201C092210192E11DC08330D1F482
:107D4000F7018281882331F43092220120922101AF
:107D500094E011C0813031F450922201409221010F
:107D60009CE109C0823031F47092220160922101BD
:107D70009EE001C090E0F0E4F0930B0119C02830C0
:107D800019F426E231E009C0293019F48093260164
:107D900006C02A3021F42CE131E091E003C02CE14F
:107DA00031E090E0309322012093210101C090E066
:107DB000D70117968C91882331F009C0292F80E8CC
:107DC00080930B0105C0F7012681291708F0292FA0
:107DD0002093010175C080910B0187FF71C08091D4
:107DE0000E01192F891708F4182F811B80930E019B
:107DF00000E0882309F401E080911001873010F041
:107E0000E70115C050910F01E0910C01F0910D01B7
:107E100040E04BC080910C0190910D010196909330
:107E20000D0180930C01019769910E94FF3F9E0113
:107E30002E19211778F340C0CF018F779070892BCE
:107E400049F4F89433E030935700E895789407B6F6
:107E500000FCFDCF4E5FF894D7018D919D917D017F
:107E6000B1E00C01B0935700E895112478949F017C
:107E70002E5F3F4FC9018F779070892B31F000231F
:107E800099F0411788F0552379F0F89485E08093B4
:107E90005700E895789407B600FCFDCFF89491E17F
:107EA00090935700E8957894F901411708F4C4CFEE
:107EB000F0930D01E0930C01002311F010920101E9
:107EC000109223018091000184FF80C08091010104
:107ED0008F3F09F47BC0182F893008F018E0811B10
:107EE000809301018091130198E889278093130101
:107EF000112309F458C080910B0187FF2BC080919A
:107F00000E01811708F4182F811B80930E01009138
:107F10001001C4E1D1E0E12EFF24EC0EFD1E16C0DD
:107F2000E0910C01F0910D01073020F0CF010E948B
:107F3000F73F01C084918883219680910C01909134
:107F40000D01019690930D0180930C01CE15DF0574
:107F500039F727C0209121013091220186FF0DC001
:107F6000A4E1B1E080E090E0F901E80FF91FE491AD
:107F7000ED9301961817C1F708C0D901912FE4E1DC
:107F8000F1E08D9181939150E1F71150812F90E0B4
:107F90001F5F0196820F931F90932201809321010E
:107FA00002C0193068F484E191E0612F0E94913C95
:107FB000612F6C5F6C3041F08FEF8093010104C042
:107FC0008FEF809301016EE16093000194E189B12C
:107FD000847831F49150D9F71092240110921E0147
:107FE00080910601882309F408CE0E94A93DF999E1
:107FF000FECF92BD81BDF89A992780B50895262FAE
:10800000F999FECF1FBA92BD81BD20BD0FB6F8947D
:0E801000FA9AF99A0FBE01960895F894FFCFE0
:06801E005AFF1E950F0041
:040000030000780081
:00000001FF
